:1000000019C033C032C031C030C02FC02EC02DC087
:100010002CC02BC0F8C129C086C1DEC126C025C0B6
:1000200024C023C022C021C020C01FC01EC01DC0CC
:100030001CC01BC011241FBECFEFD2E0DEBFCDBF5E
:1000400011E0A0E0B1E0E0E9FCE002C005900D9213
:10005000A431B107D9F711E0A4E1B1E001C01D92CC
:10006000AD34B107E1F7CCD211C6CACFF894809174
:100070001A018093480180911B018093490180916E
:100080001C0180934A0180911D0180934B0178945B
:10009000089510921A0110921B0110921C011092E7
:1000A0001D01089510921A0110921B0110921C015B
:1000B00010921D01DBDF089580931A0180931B01CC
:1000C00080931C0180931D01D1DF089588E7809300
:1000D0001A019CE590931B019CE190931C01809375
:1000E0001D01C4DF0895BF92CF92DF92EF92FF927D
:1000F0000F931F93CF93DF93162F072FF82EE92E20
:10010000A8019701652F742F832F922F20E030E0F4
:10011000A90106D4882319F4DD24D394A6C0A8012C
:100120009701652F742F832F922F20E030E04AE74C
:1001300054E445D587FF03C0DD24D39421C0A80132
:100140009701652F742F832F922F2FE632E143E81A
:100150005AE339D5162F072FF82EE92EDD2410C0CB
:10016000A8019701652F702F832F9E2D20E030E08E
:100170004AE754E428D5162F072FF82EE92ED394FA
:10018000A8019701652F702F832F9E2D20E030E06E
:1001900040E85FE3C5D387FDE3CFCC2410C0A801BE
:1001A0009701652F702F832F9E2D2DEC3CEC4CEC8E
:1001B0005DE309D5162F072FF82EE92EC394A80169
:1001C0009701652F702F832F9E2D20E030E040E2B5
:1001D00051E4F5D487FFE3CFA8019701652F702F75
:1001E000832F9E2D2FE632E143E05AE335D3162FBD
:1001F000072FF82EE92EA8019701652F742F832F62
:10020000922F20E030E040E251E4D9D48823ACF0D2
:10021000A8019701652F742F832F922F2DEC3CECB2
:100220004CEC5DE3D0D4162F072FF82EE92EC394A3
:1002300082E08C1514F4DA94CC24A1E0AD158CF096
:1002400015C0A8019701652F702F832F9E2D2DECCF
:100250003CEC4CEC5DE3B7D4162F072FF82EE92EBB
:10026000C394B2E0BC156CF7DA94CC24CAE1D1E0B7
:10027000BB24A8019701652F702F832F9E2DBCD31F
:10028000862F992787FD9095BC1469F4EB2DFF27E5
:10029000E7FDF095E65EFE4F8C5F9E4FDC018C9192
:1002A0008068808305C08C5F9E4FFC0180818883BD
:1002B000B3942196F4E0BF16C9F0772767FD7095D7
:1002C000872F972FCCD39B01AC01D801F7016B2F5F
:1002D000702F8F2F9E2DBFD220E030E040E251E4FE
:1002E00072D4162F072FF82EE92EC3CFBFDEDD20E4
:1002F00011F4409A01C04098DF91CF911F910F9166
:10030000FF90EF90DF90CF90BF90089581E88093A9
:10031000810080E593EC90938B0080938A0085E2C6
:1003200080936F0008951F920F920FB60F921124C1
:100330002F933F934F938F939F93EF93FF938091CE
:100340008A0090918B00805B9C4390938B008093FC
:100350008A0078941BB888B18E6188B99091190190
:10036000292F30E0F901E85BFE4F80818BB948B15D
:1003700020503F4FF90180818095842388B9892FCF
:100380008F5F80931901843010F0109219018091D1
:1003900022019091230101969093230180932201E1
:1003A0008091390190914B01882339F08091390176
:1003B000815080933901906801C09F7790934B01E1
:1003C000FF91EF919F918F914F913F912F910F90BE
:1003D0000FBE0F901F9018951F920F920FB60F929D
:1003E00011248F939F938091420190914301019634
:1003F00090934301809342019F918F910F900FBE84
:100400000F901F9018951F920F920FB60F92112404
:100410002F933F938F939F93AF93BF938091150139
:1004200090911601A0911701B09118010196A11D9C
:10043000B11D8093150190931601A0931701B093FD
:10044000180120914C01213069F58093340190937B
:100450003501A0933601B093370120918600309189
:10046000870030933F0120933E012091420130915B
:1004700043013093410120934001B09B10C0209173
:100480003E0130913F0137FD0AC02091400130917B
:1004900041012F5F3F4F309341012093400122E003
:1004A00020934C01B59B0DC00196A11DB11D8093F9
:1004B000150190931601A0931701B093180180E2E3
:1004C00086BBBF91AF919F918F913F912F910F90DC
:1004D0000FBE0F901F901895F999FECF81BDF89A25
:1004E00080B50895F999FECF61BDF89A90B5891746
:1004F00031F0F89461BD80BDFA9AF99A7894089524
:100500000F931F93DF93CF930F92CDB7DEB78B017D
:100510009983E8DFB8016F5F7F4F9981892FE2DF10
:100520000F90CF91DF911F910F910895F999FECF10
:1005300081BDF89A40B5F999FECF019681BDF89A30
:1005400080B5382F20E0240F311DC9010895CF92C6
:10055000DF92EF92FF921F93CF93DF9313B1109529
:100560001470809114018095812309F43FC0C090DC
:100570001E01D0901F01E0902001F0902101C701E1
:10058000B60127E73EEB4FE75FE319D3181674F582
:10059000C701B60125EC30E240E85FE3C1D1882312
:1005A0002CF58091440190914501A0914601B091B4
:1005B0004701EC01C050DD42BE01882777FD8095E0
:1005C000982F6050734D8E4C9E4F49D260933001EE
:1005D0007093310180933201909333018FEF6CDD82
:1005E000CE0162E070E08CDF1092380110931401AC
:1005F000DF91CF911F91FF90EF90DF90CF90089502
:100600008F929F92AF92BF92CF92DF92EF92FF9222
:100610000F931F93CF93DF9380E880936100109234
:10062000610085E085B91BB88FEF8AB988B18E6308
:1006300088B98FE187B9459A10924C011092380120
:1006400082E090E073DF9C01B901882777FD8095F7
:10065000982F6050734D8E4C9E4F01D260933001A5
:1006600070933101809332019093330181E880933C
:10067000810080E593EC90938B0080938A0085E263
:1006800080936F0080E418DD789411E002E4F89420
:1006900080914C01882369F480912201909123017B
:1006A0008538910530F010934C011092230110927F
:1006B0002201C0912201D0912301789480914C01B4
:1006C000823009F0B7C080914001909141012091A2
:1006D0003E0130913F01A0E0B0E0DC01992788277E
:1006E00040E050E0820F931FA41FB51F80933A0192
:1006F00090933B01A0933C01B0933D0180913A015E
:1007000090913B01A0913C01B0913D0120912401C9
:10071000309125014091260150912701821B930BB6
:10072000A40BB50B8093440190934501A09346011F
:10073000B093470180913A0190913B01A0913C0117
:10074000B0913D018093240190932501A09326014F
:10075000B09327018091340190913501A091360129
:10076000B0913701209128013091290140912A014F
:1007700050912B01821B930BA40BB50B80932C0182
:1007800090932D01A0932E01B0932F0180913401FD
:1007900090913501A0913601B091370180932801E5
:1007A00090932901A0932A01B0932B0110924C0140
:1007B000809138018823E1F160912C0170912D0125
:1007C00080912E0190912F01C0904401D09045015D
:1007D000E0904601F090470140D1209130013091E6
:1007E00031014091320150913301EDD14B015C0157
:1007F000C701B60132D19B01AC01C501B40194D04F
:10080000262F372F482F592F20931E0130931F0179
:100810004093200150932101359905C020E030E03C
:1008200040E752E4D0D15FDC0093390190DE02C092
:10083000109338013FE0C13AD30708F428CF46DCD3
:100840001092380110924C01F894109223011092EA
:10085000220178941CCF5058BB27AA270ED075C10F
:1008600066D130F06BD120F031F49F3F11F41EF4CB
:100870005BC10EF4E095E7FB51C1E92F77D180F31E
:10088000BA17620773078407950718F071F49EF58D
:100890008FC10EF4E0950B2EBA2FA02D0B01B901DC
:1008A00090010C01CA01A0011124FF27591B99F0E6
:1008B000593F50F4503E68F11A16F040A22F232FF2
:1008C000342F4427585FF3CF469537952795A79542
:1008D000F0405395C9F77EF41F16BA0B620B730BE9
:1008E000840BBAF09150A1F0FF0FBB1F661F771F5A
:1008F000881FC2F70EC0BA0F621F731F841F48F40F
:10090000879577956795B795F7959E3F08F0B3CF94
:100910009395880F08F09927EE0F9795879508957E
:10092000D9D008F481E008950CD00FC107D140F070
:10093000FED030F021F45F3F19F0F0C0511139C101
:10094000F3C014D198F39923C9F35523B1F3951B40
:10095000550BBB27AA2762177307840738F09F5FE0
:100960005F4F220F331F441FAA1FA9F333D00E2E4F
:100970003AF0E0E830D091505040E695001CCAF7BC
:1009800029D0FE2F27D0660F771F881FBB1F261781
:1009900037074807AB07B0E809F0BB0B802DBF0154
:1009A000FF2793585F4F2AF09E3F510568F0B6C06D
:1009B00000C15F3FECF3983EDCF386957795679531
:1009C000B795F7959F5FC9F7880F911D9695879505
:1009D00097F90895E1E0660F771F881FBB1F621724
:1009E00073078407BA0720F0621B730B840BBA0BE2
:1009F000EE1F88F7E095089504D06894B111D9C02E
:100A00000895BCD088F09F5790F0B92F9927B7511F
:100A1000A0F0D1F0660F771F881F991F1AF0BA95C2
:100A2000C9F712C0B13081F0C3D0B1E00895C0C0A1
:100A3000672F782F8827B85F39F0B93FCCF38695B8
:100A400077956795B395D9F73EF490958095709515
:100A500061957F4F8F4F9F4F0895E89409C097FB92
:100A60003EF490958095709561957F4F8F4F9F4F85
:100A70009923A9F0F92F96E9BB279395F6958795C9
:100A800077956795B795F111F8CFFAF4BB0F11F48C
:100A900060FF1BC06F5F7F4F8F4F9F4F16C0882333
:100AA00011F096E911C0772321F09EE8872F762F69
:100AB00005C0662371F096E8862F70E060E02AF0AA
:100AC0009A95660F771F881FDAF7880F9695879596
:100AD00097F90895990F0008550FAA0BE0E8FEEF6B
:100AE00016161706E807F907C0F012161306E407F2
:100AF000F50798F0621B730B840B950B39F40A26EB
:100B000061F0232B242B252B21F408950A2609F4C8
:100B1000A140A6958FEF811D811D089597F99F67CC
:100B200080E870E060E008959FEF80EC0895002475
:100B30000A941616170618060906089500240A9442
:100B400012161306140605060895092E0394000CC8
:100B500011F4882352F0BB0F40F4BF2B11F460FF57
:100B600004C06F5F7F4F8F4F9F4F089557FD905880
:100B7000440F551F59F05F3F71F04795880F97FB61
:100B8000991F61F09F3F79F087950895121613061B
:100B90001406551FF2CF4695F1DF08C0161617064A
:100BA0001806991FF1CF869571056105089408957F
:100BB000E894BB2766277727CB0197F908958ADF4A
:100BC00008F48FEF08950BD0C0CFB1DF28F0B6DF67
:100BD00018F0952309F0A2CFA7CF1124EACFC6DFE2
:100BE000A0F3959FD1F3950F50E0551F629FF00140
:100BF000729FBB27F00DB11D639FAA27F00DB11D99
:100C0000AA1F649F6627B00DA11D661F829F222721
:100C1000B00DA11D621F739FB00DA11D621F839FA8
:100C2000A00D611D221F749F3327A00D611D231F7E
:100C3000849F600D211D822F762F6A2F11249F57CC
:100C400050408AF0E1F088234AF0EE0FFF1FBB1FEF
:100C5000661F771F881F91505040A9F79E3F51058E
:100C600070F05CCFA6CF5F3FECF3983EDCF3869547
:100C700077956795B795F795E7959F5FC1F7FE2B39
:100C8000880F911D9695879597F90895F894FFCF51
:100C9000100804023F065B4F666D7D077F6F777C0F
:040CA000395E7971CF
:00000001FF
